:1000000000308A00C8290000FF00030E8301A10010
:100010007F08A0000A08A8008A01A00E0408A20018
:100020007708A3007808A4007908A5007A08A6003C
:100030007B08A700831383128C308400801D222844
:100040008C1939288B1E26280B193B28220884007E
:100050002308F7002408F8002508F9002608FA000C
:100060002708FB0028088A00210E8300FF0E7F0E60
:1000700009008A1189288A11B7280A108A100A11E2
:100080008207023406340E341E343E347E34FE348D
:10009000FF340A108A100A1182070A345034573488
:1000A0004D343A34253430343334753420345234BA
:1000B00055344E343A3425343034333475340034C6
:1000C0000A108A100A1182070A34523455344E3409
:1000D0003A3420342534333475346D347334203459
:1000E00000340A108A100A1182070A3441344C3451
:1000F00047343A342534303433347534203425349D
:10010000303433347534203425343034333475345A
:1001100000342A0893008C118A112628C408031D74
:100120009D288316061183120611831694018312EB
:10013000940183168C11B52883124408073C0318D8
:10014000A3280830C400C40344083D20F800AA00D6
:10015000831606118312061183169401223083122E
:1001600094002A08930083168C15831200342B0800
:100170002C040319BF282B080319AC03AB03AD08EB
:10018000031DAD03AF080319D2282F08073C031C39
:10019000D228AD08031DD2282E08AD00AF0A2F08C3
:1001A000C4008E200B118A11262883160108C0393D
:1001B0000138810083128B16C0308B048A11EF291D
:1001C0003D08043C031DE82883168610831286141C
:1001D000303083169F0083123D0DF700F70DF70DA9
:1001E000F830F7057708413E9F0064001030F700B3
:1001F000F70BF828000000001F1564001030F7000E
:10020000F70B002900000000831686108312861069
:100210001E08F800003483169818102983120B2941
:1002200083124108990000344208F8014102031882
:100230001C294108F7002829F7010830C300C10D27
:10024000F70D420877020318F700F80DC30B1F29BA
:1002500000344013C0123F08C1006430C2001421B2
:100260007708BF007808031D5329C01A5329C01905
:100270006129401B41294018412940194129C01BCF
:100280006129401C4D29C01B6129401B4D29401884
:10029000612940194D29C01B61292030401E303092
:1002A000C1000B216129C016C01F5D29780880009C
:1002B000F8002D30C1000B21C01330307807C10089
:1002C0000B21401B6C293F08C1000A30C2001421D9
:1002D0007708BF0040173229C01F71292D30C10097
:1002E0000B2130303F07C1000B2100343D3084002A
:1002F000000803198C290130F800BF30F7006400B2
:10030000F70B7F29F80B7D295830F700F70B86296A
:1003100000006400800B7B290034A9018B1BA91706
:100320008B133D08C4008E20A91B8B17C0308B0493
:1003300000348B123E08AC003D08AB008B16003435
:100340008B12AB08031DA729AC080319A92900309B
:10035000AA290130F8007818AF293D10B0293D14C2
:100360008B1600303D180130F80000348B1201303C
:10037000AF003D08AE002E08AD008B16A9018B1B07
:10038000A9178B130130C4008E20A91B8B170034D2
:1003900084011F30830583161F129F121B088039AA
:1003A0009B0007309C00050864001C0883120D1395
:1003B000623083168F001F30920004308312920047
:1003C0000C30970095018316861183128611143024
:1003D00095000B138B138B1BEA29ED29D5280330CD
:1003E000B000300B2C2A6400BD01E0207808B20078
:1003F000B20CB20C3F30B2050130BD00E0207808ED
:10040000B300B30E0F30B305BD013D084920BD0A4E
:10041000F700C1000B2105303D02031D052A3208FB
:10042000BF00C00129210930BE003E084920BE0A94
:10043000F700C1000B210E303E02031D152A3308C0
:10044000BF00C00129211430BD007621320895007B
:100450003308BD008D21F3293008023C031D7D2A9D
:10046000B5010130BD00E0207808B400BD013D08B1
:100470006020BD0AF700C1000B2106303D02031DBC
:10048000372A3408BF001030C00029216D30C10068
:100490000B217330C1000B212030C1000B210A3029
:1004A000BD007621B508031D5B2AB50A0730BE00E2
:1004B000D030BD009921350B6D2AA021F808031911
:1004C0006D2AB50A5230C1000B213408BD00B62197
:1004D0000730BE00D030BD0099213508023C031D15
:1004E0007B2AA021F80803197B2AB50A5330C100E2
:1004F0000B21BD018D216400312A3008033C031D0E
:10050000DB2AB6016400BD01E0207808B700BD0118
:10051000E0200310780C323EB7000430BD00E0202C
:100520007808B8003708380203189A2A36081D3CA4
:100530000318B60A37083802031CA12AB608031D9F
:10054000B6030A30B807370838020318AB2A360852
:100550001D3C0318B60A3608183C0318B12A183097
:10056000B6001430B600360895000B138B138B1BA6
:10057000B62AB92ABD013D087120BD0AF700C100A5
:100580000B2105303D02031DBB2A3708BF00C00107
:1005900029212030C1000B213808BF00C0012921CA
:1005A0002030C1000B213608BF00C00129210A30CC
:1005B000BD007621822AB008031D412BB9013630D7
:1005C000BE00B030BD0099213C146400BD01E020A4
:1005D0007808BA00BD01E0200310780C323EBA0062
:1005E0000430BD00E0207808BB003A083B02031845
:1005F000FD2A39081D3C0318B90A3A083B02031CBE
:10060000042BB908031DB9030A30BB073A083B02A3
:1006100003180E2B39081D3C0318B90A3908183C79
:100620000318142B1830B90039089500BD013D0896
:100630007120BD0AF700C1000B2105303D02031DEA
:10064000172B3A08BF00C00129212030C1000B211F
:100650003B08BF00C00129212030C1000B2139080F
:10066000BF00C00129210A30BD007621A021F80871
:100670000319402B3C1C402B3C104130BD00B621DF
:04068000E52A630004
:04400E00382FFF3F09
:00000001FF
